:100000008D2964001720031801285620A801083004
:10001000A300572017200318A80AAB1EA801A20CA2
:10002000A30B0928AB1AA2135720220808003A088C
:100030008400380884178004841300052B1B3806BD
:10004000FF3E08000408A6003A088400F030B70517
:100050000830A70003100318B70A3C20A60CA70B12
:100060002B280000AB1A370C3C208B2103143C20BA
:100070002F08A3002E08EC288413AB1F4B28000880
:1000800038042B1F38068000841700083804031C2E
:1000900038068000572800083804031C38062B1B3C
:1000A00038068000841738098005572837172B0831
:1000B0001F39FF3EA1002A08F53E0318A10A371F89
:1000C000F9283713A00002302B21F928B71329088B
:1000D0000319B7170530A8002730A30010307C2083
:1000E0000330A300E8307C20A30164307C20A3010E
:1000F0000A307C2024088328A2002508A1002408B7
:10010000A00051212008A000A8030319B713290853
:1001100003198D282802031808002008031DB713AF
:10012000B71B0800303E83290830A60037180D2180
:100130003B08840039083719B720371DB9203A0821
:1001400084003809BD203A088400A10CA00C0008E6
:100150003804031C38068000B020A60BA328882989
:100160003B088400390880060000800608008004EF
:10017000BC28FF3A8005BD28FF3A841780058829EE
:10018000A000A00DA00DA00D3830A00581302004E6
:100190009F000030A1003230F9201F151F19CE2812
:1001A0001E08A10083161E08882903178D008316D8
:1001B0008C130C1483120C08882903178C008316E7
:1001C0008C130C1555308D00AA308D008C148C18B2
:1001D000E7280C118829A301A200FF30A207031C05
:1001E000A307031C88290330A100DF30F920ED2884
:1001F000A101E83EA000A109FC30031C0229A007D0
:100200000318FF28A0076400A10FFF282018082961
:10021000A01C0C2900000C290800A400A201A301C5
:100220001529A10CA00CA20DA30DFF3E0318112946
:10023000240823212208A0042308A1042008080080
:100240000310A00DA10DFF3E0318202920088829C6
:100250000310A10CA00CFF3E0318282920088829B0
:10026000A101A301A20001303A29A101A301A2002A
:1002700004303A29A80023082102031D412922083D
:100280002002043003180130031902302805031D31
:10029000FF3088290038031DFF300405031DFF309F
:1002A00088291030A600A501A401210DA40DA50DDB
:1002B0002208A4022308031C230FA50203186729A0
:1002C0002208A40723080318230FA5070310A00D75
:1002D000A10DA60B5529200888291030A800A101DE
:1002E000A001A70CA60C031C7B292208A007230849
:1002F0000318230FA107A10CA00CA50CA40CA80B9C
:10030000712924088829840031088A003008820075
:100310008313031383126400080083161F308500C3
:100320000130860002308700831281309F008316DF
:1003300084309F008312871583168711073083123C
:10034000BA000230B8005430AA004030AB00AE0111
:10035000AF012A308A01232020308A012320523025
:100360008A01232058308A01232020308A0123204B
:1003700031308A01232033308A01232037308A012B
:1003800023202D308A01232031308A01232033306D
:100390008A01232038308A01232020308A0123203B
:1003A0004D308A01232048308A0123207A308A0187
:1003B00023202E308A01232020308A01232056302A
:1003C0008A01232020308A01232031308A01232012
:1003D0002E308A01232030308A01232020308A01E8
:1003E000232045308A01232041308A0123203330E5
:1003F0008A01232043308A0123204E308A012320A2
:100400004F308A01232020308A0123202A308A019C
:1004100023200A308A0123200D308A01232007304F
:10042000BA000230B8005430AA004030AB00AE0130
:10043000AF012D308A0123202D308A0123202D3059
:100440008A0123202D308A0123202D308A01232088
:100450002D308A0123202D308A0123202D308A015E
:1004600023202D308A0123202D308A0123202D3096
:100470008A0123202D308A0123202D308A01232058
:100480002D308A0123202D308A0123202D308A012E
:1004900023202D308A0123202D308A0123202D3066
:1004A0008A0123202D308A0123202D308A01232028
:1004B0002D308A0123202D308A0123202D308A01FE
:1004C00023202D308A0123202D308A0123202D3036
:1004D0008A0123202D308A0123202D308A012320F8
:1004E0002D308A0123202D308A0123202D308A01CE
:1004F00023200A308A0123200D308A01232007306F
:10050000A300D0308A01EC2000308A01D520DE0023
:1005100001308A01D520E20002308A01D520E100B5
:100520008A150A124C2764308A01EB2064005E08A9
:10053000013C8A150A120319BB2B64005E08023CB9
:100540008A150A120319D52B64005E08033C8A152C
:100550000A120319EF2B64005E08043C8A150A1284
:100560000319092C64005E08053C8A150A12031958
:10057000232C64005E08063C8A150A1203193E2CDF
:100580000730BA000230B8005430AA004030AB0047
:10059000AE01AF012D308A0123202D308A012320A6
:1005A0002D308A0123202D308A0123202D308A010D
:1005B00023202D308A0123202D308A0123202D3045
:1005C0008A0123202D308A0123202D308A01232007
:1005D0002D308A0123202D308A0123202D308A01DD
:1005E00023202D308A0123202D308A0123202D3015
:1005F0008A0123202D308A0123202D308A012320D7
:100600002D308A0123202D308A0123202D308A01AC
:1006100023202D308A0123202D308A0123202D30E4
:100620008A0123202D308A0123202D308A012320A6
:100630002D308A0123202D308A0123202D308A017C
:1006400023202D308A0123202D308A0123202D30B4
:100650008A0123202D308A0123202D308A01232076
:100660002D308A0123202D308A0123202D308A014C
:1006700023202D308A0123202D308A0123202D3084
:100680008A0123202D308A0123202D308A01232046
:100690002D308A0123202D308A0123202D308A011C
:1006A00023202D308A0123202D308A0123202D3054
:1006B0008A0123202D308A0123202D308A01232016
:1006C0002D308A0123202D308A0123202D308A01EC
:1006D00023202D308A0123202D308A0123202D3024
:1006E0008A0123202D308A0123202D308A012320E6
:1006F0002D308A0123202D308A0123202D308A01BC
:1007000023202D308A0123202D308A0123202D30F3
:100710008A0123200A308A0123200D308A012320F8
:100720000730BA000230B8005430AA004030AB00A5
:10073000AE01AF0120308A01232020308A0123201E
:1007400020308A01232020308A01232020308A0192
:10075000232020308A01232020308A0123202030CA
:100760008A01232020308A01232020308A0123207F
:1007700020308A01232020308A01232020308A0162
:10078000232020308A01232020308A01232020309A
:100790008A01232020308A01232020308A0123204F
:1007A00020308A01232020308A01232020308A0132
:1007B000232020308A01232020308A01232020306A
:1007C0008A01232020308A0123202A308A01232015
:1007D00020308A01232020308A01232043308A01DF
:1007E000232061308A0123206E308A01232061306A
:1007F0008A0123206C308A01232065308A0123205E
:1008000073308A01232020308A01232052308A014C
:10081000232058308A01232020308A0123202030D1
:100820008A0123202A308A01232020308A012320B4
:1008300020308A01232020308A01232020308A01A1
:10084000232020308A01232020308A0123202030D9
:100850008A01232020308A01232020308A0123208E
:1008600020308A01232020308A01232020308A0171
:10087000232020308A01232020308A0123202030A9
:100880008A01232020308A01232020308A0123205E
:1008900020308A01232020308A01232020308A0141
:1008A000232020308A01232020308A012320203079
:1008B0008A0123200A308A0123200D308A01232057
:1008C0000730BA000230B8005430AA004030AB0004
:1008D000AE01AF0143308A01232048308A01232032
:1008E0002D308A01232031308A01232020308A01D3
:1008F000232031308A01232033308A0123203730EE
:100900008A0123202E308A01232031308A012320BE
:1009100030308A01232030308A0123202E308A0192
:10092000232030308A01232020308A0123204D30BB
:100930008A01232048308A0123207A308A0123202B
:1009400020308A01232020308A01232043308A016D
:10095000232048308A0123202D308A012320323081
:100960008A01232020308A01232031308A0123206C
:1009700033308A01232037308A0123202E308A0128
:10098000232033308A01232030308A012320303065
:100990008A0123202E308A01232030308A0123202F
:1009A00020308A0123204D308A01232048308A01DB
:1009B00023207A308A01232020308A01232020300E
:1009C0008A01232043308A01232048308A012320D2
:1009D0002D308A01232033308A01232020308A01E0
:1009E000232031308A01232033308A0123203730FD
:1009F0008A0123202E308A01232034308A012320CB
:100A000030308A01232030308A0123202E308A01A1
:100A1000232030308A01232020308A0123204D30CA
:100A20008A01232048308A0123207A308A0123203A
:100A30000A308A0123200D308A0123200730BA00B2
:100A40000230B8005430AA004030AB00AE01AF0114
:100A500043308A01232048308A0123202D308A0127
:100A6000232034308A01232020308A012320313092
:100A70008A01232033308A01232037308A01232042
:100A80002E308A01232035308A01232030308A011C
:100A9000232030308A0123202E308A012320303059
:100AA0008A01232020308A0123204D308A0123200F
:100AB00048308A0123207A308A01232020308A019D
:100AC000232020308A01232043308A01232048300C
:100AD0008A0123202D308A01232035308A012320EA
:100AE00020308A01232031308A01232033308A01CB
:100AF000232037308A0123202E308A0123203630EC
:100B00008A01232032308A01232030308A012320B9
:100B10002E308A01232030308A01232020308A01A0
:100B200023204D308A01232048308A0123207A3047
:100B30008A01232020308A01232020308A012320AB
:100B400043308A01232048308A0123202D308A0136
:100B5000232036308A01232020308A01232031309F
:100B60008A01232033308A01232037308A01232051
:100B70002E308A01232039308A01232031308A0126
:100B8000232032308A0123202E308A012320353061
:100B90008A01232020308A0123204D308A0123201E
:100BA00048308A0123207A308A0123200A308A01C2
:100BB00023200D308A0123200730BA000230B8000C
:100BC0005430AA004030AB00AE01AF012A308A0198
:100BD000232052308A01232058308A0123202030DC
:100BE0008A01232061308A01232063308A01232077
:100BF00074308A01232075308A01232061308A01F4
:100C000023206C308A01232020308A0123204330A6
:100C10008A01232048308A0123202D308A01232095
:100C20000130A9005E08A400A5012230B000B10186
:100C30008A0166202A308A01232020308A0123205D
:100C400043308A01232061308A0123206D308A01DC
:100C5000232062308A01232069308A0123206F30EB
:100C60008A01232020308A01232064308A01232036
:100C700065308A01232020308A01232063308A01D5
:100C8000232061308A0123206E308A0123206130C5
:100C90008A0123206C308A0123203D308A012320E1
:100CA00063308A01232020308A01232020308A01EA
:100CB00023204D308A01232065308A0123206E30A5
:100CC0008A01232075308A0123202D308A012320B8
:100CD00052308A01232058308A0123203D308A0176
:100CE00023206D308A0123200A308A0123200D3011
:100CF0008A0123200730BA000230B8005430AA001D
:100D00004030AB00AE01AF012D308A0123202D30E1
:100D10008A0123202D308A0123202D308A012320AF
:100D20002D308A0123202D308A0123202D308A0185
:100D300023202D308A0123202D308A0123202D30BD
:100D40008A0123202D308A0123202D308A0123207F
:100D50002D308A0123202D308A0123202D308A0155
:100D600023202D308A0123202D308A0123202D308D
:100D70008A0123202D308A0123202D308A0123204F
:100D80002D308A0123202D308A0123202D308A0125
:100D900023202D308A0123202D308A0123202D305D
:100DA0008A0123202D308A0123202D308A0123201F
:100DB0002D308A0123202D308A0123202D308A01F5
:100DC00023202D308A0123202D308A0123202D302D
:100DD0008A0123202D308A0123202D308A012320EF
:100DE0002D308A0123202D308A0123202D308A01C5
:100DF00023202D308A0123202D308A0123202D30FD
:100E00008A0123202D308A0123202D308A012320BE
:100E10002D308A0123202D308A0123202D308A0194
:100E200023202D308A0123202D308A0123202D30CC
:100E30008A0123202D308A0123202D308A0123208E
:100E40002D308A0123202D308A0123202D308A0164
:100E500023202D308A0123202D308A0123202D309C
:100E60008A0123202D308A0123202D308A0123205E
:100E70002D308A0123202D308A0123202D308A0134
:100E800023202D308A0123200A308A0123200D30AF
:100E90008A0123200730BA000130B8005430AA007C
:100EA0004030AB008A010120E0006008A0006430FF
:100EB0008A013521B2006008A00062308A01302129
:100EC000B4003208840034088A014A218A110A12C7
:100ED000031D842F6008A0006E308A013521B20006
:100EE0006008A0006C308A013021B4003208840010
:100EF00034088A014A218A150A12031D9D2964308B
:100F00008A01EB208A01C02A0730BA000230B800FB
:100F10005430AA004030AB00AE01AF0149308A0125
:100F200023206E308A01232074308A0123207230FE
:100F30008A0123206F308A01232064308A01232014
:100F400075308A01232063308A01232069308A01A9
:100F5000232072308A01232020308A0123204E3042
:100F60008A012320BA308A01232020308A012320DD
:100F700063308A01232061308A0123206E308A0188
:100F8000232061308A0123206C308A0123203A30EB
:100F90008A0123205F308A01232020308A01232008
:100FA00020308A01232020308A01232020308A012A
:100FB000232020308A01232020308A012320203062
:100FC0008A01232020308A01232020308A01232017
:100FD00020308A01232020308A01232020308A01FA
:100FE000232020308A01232020308A012320203032
:100FF0008A01232020308A01232020308A012320E7
:1010000020308A01232020308A01232020308A01C9
:10101000232020308A01232020308A012320203001
:101020008A01232020308A01232020308A012320B6
:1010300020308A01232020308A01232020308A0199
:10104000232020308A01232020308A0123202030D1
:101050008A01232020308A01232020308A01232086
:1010600020308A01232020308A01232020308A0169
:10107000232020308A01232020308A0123202030A1
:101080008A0123200A308A0123200D308A0123207F
:101090000730BA000230B8005430AA004030AB002C
:1010A000AE01AF012D308A0123202D308A0123208B
:1010B0002D308A0123202D308A0123202D308A01F2
:1010C00023202D308A0123202D308A0123202D302A
:1010D0008A0123202D308A0123202D308A012320EC
:1010E0002D308A0123202D308A0123202D308A01C2
:1010F00023202D308A0123202D308A0123202D30FA
:101100008A0123202D308A0123202D308A012320BB
:101110002D308A0123202D308A0123202D308A0191
:1011200023202D308A0123202D308A0123202D30C9
:101130008A0123202D308A0123202D308A0123208B
:101140002D308A0123202D308A0123202D308A0161
:1011500023202D308A0123202D308A0123202D3099
:101160008A0123202D308A0123202D308A0123205B
:101170002D308A0123202D308A0123202D308A0131
:1011800023202D308A0123202D308A0123202D3069
:101190008A0123202D308A0123202D308A0123202B
:1011A0002D308A0123202D308A0123202D308A0101
:1011B00023202D308A0123202D308A0123202D3039
:1011C0008A0123202D308A0123202D308A012320FB
:1011D0002D308A0123202D308A0123202D308A01D1
:1011E00023202D308A0123202D308A0123202D3009
:1011F0008A0123202D308A0123202D308A012320CB
:101200002D308A0123202D308A0123200A308A01C3
:1012100023200D308A01232032308A01EB20073051
:10122000BA000130B8005430AA004030AB008A0147
:101230000120E0006008A00032308A013521B200B0
:101240006008A00030308A013021B40032088400E8
:1012500034088A014A218A150A12031DBB2B600833
:10126000A00033308A013521B2006008A00031307F
:101270008A013021B4003208840034088A014A21EE
:101280008A150A12031DD52B6008A00034308A018C
:101290003521B2006008A00032308A013021B4004C
:1012A0003208840034088A014A218A150A12031D73
:1012B000EF2B6008A00035308A013521B2006008AC
:1012C000A00033308A013021B40032088400340891
:1012D0008A014A218A150A12031D092C6008A00000
:1012E00036308A013521B2006008A00034308A010E
:1012F0003021B4003208840034088A014A218A155A
:101300000A12031D232C6008A00037308A01352102
:10131000B2006008A00035308A013021B4003208E4
:10132000840034088A014A218A150A12031D3E2CC2
:1013300064308A01EB208A01C02A64308A01EB20E4
:101340000730BA000230B8005430AA004030AB0079
:10135000AE01AF012A308A0123204D308A012320BB
:1013600045308A0123204E308A01232055308A01DE
:1013700023202D308A01232052308A012320583027
:101380008A0123202A308A01232020308A01232049
:1013900043308A01232048308A0123202D308A01DE
:1013A00023200130A9005E08A400A5012230B0006E
:1013B000B1018A01662020308A01232020308A0171
:1013C000232076308A0123203D308A0123205630A5
:1013D0008A0123206F308A0123206C308A01232068
:1013E00075308A0123206D308A01232065308A01FF
:1013F00023206E308A01232020308A0123202030D0
:101400008A01232071308A0123203D308A01232064
:1014100053308A01232071308A01232075308A01DC
:10142000232065308A0123206C308A012320633019
:101430008A01232068308A01232020308A0123205A
:1014400020308A0123206E308A0123203D308A011A
:1014500023204E308A01232069308A0123207630F0
:101460008A01232065308A0123206C308A012320E1
:101470002D308A01232052308A01232058308A01DE
:10148000232020308A01232020308A01232063304A
:101490008A0123203D308A01232043308A01232002
:1014A00061308A0123206E308A01232061308A0155
:1014B00023206C308A0123202D308A0123205230D2
:1014C0008A01232058308A0123200A308A012320F0
:1014D0000D308A0123200730BA000230B8005430A2
:1014E000AA004030AB00AE01AF012D308A012320AD
:1014F0002D308A0123202D308A0123202D308A01AE
:1015000023202D308A0123202D308A0123202D30E5
:101510008A0123202D308A0123202D308A012320A7
:101520002D308A0123202D308A0123202D308A017D
:1015300023202D308A0123202D308A0123202D30B5
:101540008A0123202D308A0123202D308A01232077
:101550002D308A0123202D308A0123202D308A014D
:1015600023202D308A0123202D308A0123202D3085
:101570008A0123202D308A0123202D308A01232047
:101580002D308A0123202D308A0123202D308A011D
:1015900023202D308A0123202D308A0123202D3055
:1015A0008A0123202D308A0123202D308A01232017
:1015B0002D308A0123202D308A0123202D308A01ED
:1015C00023202D308A0123202D308A0123202D3025
:1015D0008A0123202D308A0123202D308A012320E7
:1015E0002D308A0123202D308A0123202D308A01BD
:1015F00023202D308A0123202D308A0123202D30F5
:101600008A0123202D308A0123202D308A012320B6
:101610002D308A0123202D308A0123202D308A018C
:1016200023202D308A0123202D308A0123202D30C4
:101630008A0123202D308A0123202D308A01232086
:101640002D308A0123202D308A0123202D308A015C
:1016500023202D308A0123202D308A0123202D3094
:101660008A0123202D308A0123202D308A01232056
:101670002D308A0123202D308A0123202D308A012C
:1016800023202D308A0123202D308A0123202D3064
:101690008A0123202D308A0123202D308A01232026
:1016A0002D308A0123200A308A0123200D308A013F
:1016B00023200730BA000130B8005430AA0040306F
:1016C000AB008A010120E0006008A0006F308A01B1
:1016D0003521B2006008A0006D308A013021B400CD
:1016E0003208840034088A014A218A150A12031D2F
:1016F000302E6008A00072308A013521B2006008E7
:10170000A00070308A013021B4003208840034080F
:101710008A014A218A150A12031D442D6008A0007F
:1017200077308A013521B2006008A00075308A0147
:101730003021B4003208840034088A014A218A1515
:101740000A12031D582C6008A00064308A0135215C
:10175000B2006008A00062308A013021B400320873
:10176000840034088A014A218A110A12031DC02A02
:101770008A150A129D29E330DF00C0010230C10042
:101780008030C2002730C3008A150A12F1260130CA
:10179000DE0003178D0103135E088A01DD2005308A
:1017A0008A01EB208A150A129D29E330DF00C0016F
:1017B0000230C1009030C2002730C3008A150A12DF
:1017C000F1260230DE0003178D0103135E088A0143
:1017D000DD2005308A01EB208A150A129D29E330AD
:1017E000DF00C0010230C1009830C2002730C300C2
:1017F0008A150A12F1260330DE0003178D01031348
:101800005E088A01DD2005308A01EB208A150A1264
:101810009D29E330DF00C0010230C100A030C200CA
:101820002730C3008A150A12F1260430DE000317A0
:101830008D0103135E088A01DD2005308A01EB204B
:101840008A150A129D29E330DF008030C000023083
:10185000C1009430C2003130C3008A150A12F1264B
:101860000530DE0003178D0103135E088A01DD20B9
:1018700005308A01EB208A150A129D29E330DF002A
:10188000C0010230C100C130C2002730C3008A1538
:101890000A12F1260630DE0003178D0103135E08DD
:1018A0008A01DD2005308A01EB208A150A129D2964
:1018B0000730BA000230B8005430AA004030AB0004
:1018C000AE01AF014E308A01232069308A01232006
:1018D00076308A01232065308A0123206C308A010A
:1018E000232020308A01232056308A0123206F30A4
:1018F0008A0123206C308A01232075308A0123203D
:101900006D308A01232065308A0123206E308A01E0
:10191000232020308A0123200230A9006208A00081
:10192000A1010A30A200A3018A015121B2002108BD
:10193000B3003208A4003308A5002230B000B10182
:101940008A01662020308A01232020308A0123204A
:101950002B308A0123202F308A0123202D308A0149
:10196000232020308A01232056308A0123206F3023
:101970008A0123206C308A01232075308A012320BC
:101980006D308A01232065308A0123206E308A0160
:10199000232020308A01232020308A0123206D302B
:1019A0008A0123203D308A0123204D308A012320E3
:1019B00065308A0123206E308A01232075308A0128
:1019C00023200D308A0123200730BA000130B800EF
:1019D0005430AA004030AB008A010120E000FA3008
:1019E0008A01EB206008A0002C308A013521B2006A
:1019F0006008A0002A308A013021B4003208840037
:101A000034088A014A218A150A12031D342D600800
:101A1000A0002E308A013521B2006008A0002C30D1
:101A20008A013021B4003208840034088A014A2136
:101A30008A150A12031D3C2D6008A0006E308A0131
:101A40003521B2006008A0006C308A013021B4005A
:101A50003208840034088A014A218A150A12031DBB
:101A60009D298A150A12582C0A30E2078A150A1293
:101A70004C278A150A12582C0A30E2028A150A12DB
:101A80004C278A150A12582C0730BA000230B800C9
:101A90005430AA004030AB00AE01AF014E308A0195
:101AA000232069308A01232076308A012320653083
:101AB0008A0123206C308A01232020308A012320D0
:101AC00053308A01232071308A01232075308A0126
:101AD000232065308A0123206C308A012320633063
:101AE0008A01232068308A01232020308A012320A4
:101AF0000230A9006108A000A1010A30A200A301E0
:101B00008A015121B2002108B3003208A400330831
:101B1000A5002230B000B1018A01662020308A0180
:101B2000232020308A0123202B308A0123202F30CC
:101B30008A0123202D308A01232020308A0123208E
:101B400053308A01232071308A01232075308A01A5
:101B5000232065308A0123206C308A0123206330E2
:101B60008A01232068308A01232020308A01232023
:101B700020308A0123206D308A0123203D308A01E4
:101B800023204D308A01232065308A0123206E30C6
:101B90008A01232075308A0123200D308A012320F9
:101BA0000730BA000130B8005430AA004030AB0012
:101BB0008A010120E000FA308A01EB206008A000D1
:101BC0002C308A013521B2006008A0002A308A0139
:101BD0003021B4003208840034088A014A218A1571
:101BE0000A12031D202E6008A0002E308A01352124
:101BF000B2006008A0002C308A013021B400320805
:101C0000840034088A014A218A150A12031D282EED
:101C10006008A0006E308A013521B2006008A00083
:101C20006C308A013021B4003208840034088A0103
:101C30004A218A150A12031D9D298A150A12442D6C
:101C40000A30E1078A150A124C278A150A12442D18
:101C50000A30E1028A150A124C278A150A12442D0D
:101C60000730BA000230B8005430AA004030AB0050
:101C7000AE01AF016E308A0123203D308A0123205E
:101C80004E308A01232069308A01232076308A0170
:101C9000232065308A0123206C308A0123202030E4
:101CA0008A01232052308A01232058308A012320C0
:101CB00020308A0123202D308A0123200330A900FF
:101CC0003C08A4003D08A5002230B000B1018A0103
:101CD000662064308A01232042308A0123206D303F
:101CE0008A01232020308A0123206D308A0123209D
:101CF0003D308A0123204D308A01232065308A013E
:101D000023206E308A01232075308A0123200D3074
:101D10008A0123200730BA000130B8005430AA00ED
:101D20004030AB008A010120E0006008A0006F3065
:101D30008A013521B2006008A0006D308A0130218F
:101D4000B4003208840034088A014A218A150A1234
:101D5000031DBF2E6008A0006E308A013521B2003D
:101D60006008A0006C308A013021B4003208840081
:101D700034088A014A218A150A12031DEB2E00300D
:101D80008A01C020BE002108BF003E08A6003F080F
:101D9000A7000A30A200A3018A016D21B200250824
:101DA000B3003208A0003308A1004530A200A3010F
:101DB0008A015121B2002108B3003208823CBC00E4
:101DC0003308031C013E003CBD0064308A01EB2057
:101DD0008A150A12302EC8308A01EB208A150A12A1
:101DE0009D2986128316861206308312BA0040306F
:101DF000B8000630BB001030B9000130B7005F08F2
:101E0000A000A1018A0194208616831686120A304A
:101E100083128A01EB208612831686120630831203
:101E2000BA004030B8000630BB001030B9000130B5
:101E3000B7004008A0004108A1000F308A0195209A
:101E40008616831686120A3083128A01EB208612C8
:101E50008316861283120616831606128312061242
:101E60008316061206308312BA004030B8000630DE
:101E7000BB001030B9000130B7004208A000430891
:101E8000A1000F308A019520861683168612323003
:101E900083128A01EB20080087178316871301300D
:101EA00083128A01EB200717831607138312871604
:101EB00083168712831287128316871283120713E1
:101EC0008316071307308312BA002030B80007309A
:101ED000BB004030B9000130B7006208A000A1018A
:101EE0008A0194200730BA002030B8000730BB00C8
:101EF0004030B9000130B7006108A000A1018A019B
:101F0000942001308A01EB208713831687138312F4
:101F1000031701308D00031362088A01DD200317C7
:101F200002308D00031361088A01DD2005308A012B
:0C1F3000EB20080063008A150A129A2FAB
:02400E00753DFE
:00000001FF
